:100000000C9434000C9451000C9451000C94510049
:100010000C9451000C9451000C9451000C9451001C
:100020000C9451000C9451000C9451000C94D50385
:100030000C9458000C9451000C9451000C945100F5
:100040000C9451000C9451000C9451000C945100EC
:100050000C9451000C9451000C9451000C945100DC
:100060000C9451000C94510011241FBECFEFD8E026
:10007000DEBFCDBF11E0A0E0B1E0E2EAF9E002C0EE
:1000800005900D92A836B107D9F721E0A8E6B1E0B6
:1000900001C01D92A039B207E1F70E940E040C9432
:1000A000CF040C940000803108F08FE088BD0895E3
:1000B0001F920F920FB60F9211248F929F92AF92C0
:1000C000BF92CF92DF92EF92FF922F933F934F9385
:1000D0005F936F937F938F939F93AF93BF93EF93B0
:1000E000FF93809180008F7E8093800080E48093D6
:1000F00082008091690190916A01A0916B01B09199
:100100006C01892B8A2B8B2B81F480917E0190913D
:100110007F01A0918001B09181018093690190934A
:100120006A01A0936B01B0936C0180916901909179
:100130006A01A0916B01B0916C01009721E0A207C8
:10014000B10570F08F3FEFEF9E07E1E0AE07B1051C
:1001500050F4AC01BD01769567955795479507C05A
:10016000AC01BD0104C04FEF5FEF60E070E0841BA5
:10017000950BA60BB70B8093690190936A01A0932E
:100180006B01B0936C0120918A0030918B00240F99
:10019000351F30938B0020938A00892B8A2B8B2B61
:1001A00009F03CC110928601809173019091740115
:1001B000A0917501B0917601C0908C01D0908D0115
:1001C000E0908E01F0908F01C81AD90AEA0AFB0A62
:1001D00099F51092720180916D0190916E010097D6
:1001E000D1F0019790936E0180936D01809177011A
:1001F00090917801A0917901B0917A0180937E016C
:1002000090937F01A0938001B093810110928501AA
:100210001092840103C180917D010E94530080915E
:100220006F0082FF06C080916F008B7F80936F000C
:10023000F5C084E086BBF2C0F7FE1DC02B9880910C
:10024000730190917401A0917501B09176010197AD
:10025000A109B1098093730190937401A093750172
:10026000B0937601F094E094D094C094C11CD11C5A
:10027000E11CF11C14C02B9A8091730190917401C0
:10028000A0917501B09176010196A11DB11D8093D9
:10029000730190937401A0937501B09376018091DE
:1002A00080008061809380008091720181110FC075
:1002B00081E08093720180917B0190917C01909309
:1002C0006E0180936D0180918B010E94530080919B
:1002D0007E0190917F01A0918001B09181014091B8
:1002E0008701509188016091890170918A0184177A
:1002F0009507A607B70739F420916F013091700177
:10030000232BC9F01EC020918201309183014C0142
:100310005D0106C0880C991CAA1CBB1C369527954C
:100320008114E8E49E06A104B104A0F330937001A7
:1003300020936F01E1CF21E030E0309370012093F2
:100340006F0120918401309185014901AA2497FC15
:10035000A094BA2C8C149D04AE04BF04E4F5841759
:100360009507A607B70709F459C0E0906F01F09010
:100370007001FC01E41BF50BF7FF03C0F195E1955B
:10038000F109EE16FF0648F040937E0150937F017D
:10039000609380017093810141C0481759076A0733
:1003A0007B0778F48E199F09A109B10980937E011A
:1003B00090937F01A0938001B09381012F5F3F4F05
:1003C00029C084179507A607B70740F58E0D9F1D16
:1003D000A11DB11D15C04091770150917801609128
:1003E000790170917A0184179507A607B70780F401
:1003F00040916F0150917001840F951FA11DB11D97
:1004000080937E0190937F01A0938001B09381013E
:10041000215031093093850120938401FF91EF91A0
:10042000BF91AF919F918F917F916F915F914F910C
:100430003F912F91FF90EF90DF90CF90BF90AF90C2
:100440009F908F900F900FBE0F901F901895E1E82E
:10045000F0E01082109285001092840081E0808389
:1004600080E28093800080E098E4909389008093FC
:100470008800EFE6F0E080818260808380917701E0
:100480009091780190938B0080938A0084E086BBE2
:10049000808184608083789408959B01AC01809171
:1004A0006F0082FF06C080916F008B7F80936F008A
:1004B00002C084E086BB60E070E489E191E00E94C4
:1004C000B3042093870130938801409389015093AE
:1004D0008A0180916F00846080936F0008958093FB
:1004E0007D0160938B0108956F927F928F929F920E
:1004F000AF92BF92CF92DF92EF92FF920F931F9332
:10050000CF93DF9369017A013901DE2DCF2D621778
:1005100073078407950718F43B01D82FC92FB3013F
:100520008D2F9C2F2AE030E040E050E00E949104A3
:1005300030937C0120937B01812C30E4932E39E1B0
:10054000A32EBB24B394C501B40193014D2F5C2F9E
:100550000E949104209377013093780140937901B0
:1005600050937A0120937E0130937F014093800164
:1005700050938101C501B401A70196010E94910425
:1005800020938701309388014093890150938A0119
:10059000109383010093820184B18F6084B985B187
:1005A000836085B98AB1806D8AB95F9A5C9A5E98DA
:1005B000DF91CF911F910F91FF90EF90DF90CF903F
:1005C000BF90AF909F908F907F906F900C94270278
:1005D0008091860190917201892B08950E94E80212
:1005E0008111FCCF08950F931F9380916F0082FFBC
:1005F00006C080916F008B7F80936F0002C084E003
:1006000086BB0091730110917401209175013091A6
:10061000760180916F00846080936F00B801C901FA
:100620001F910F91089520916F0022FF06C0209125
:100630006F002B7F20936F0002C024E026BB6093E5
:100640008C0170938D0180938E0190938F0181E0D6
:100650008093860180916F00846080936F0008957D
:1006600020916F0022FF06C020916F002B7F209306
:100670006F0002C024E026BB609373017093740185
:10068000809375019093760160938C0170938D0136
:1006900080938E0190938F0181E0809386018091F9
:1006A0006F00846080936F0008950F931F93809173
:1006B0006F0082FF06C080916F008B7F80936F0078
:1006C00002C084E086BB009184011091850122273D
:1006D00017FD2095322F8091730190917401A091A4
:1006E0007501B091760140918C0150918D0160911E
:1006F0008E0170918F01481759076A077B073CF4F8
:1007000030952095109501951F4F2F4F3F4F6091C9
:100710007301709174018091750190917601600F61
:10072000711F821F931F0E94130380916F008460CA
:1007300080936F001F910F9108950F931F93209145
:100740006F0022FF06C020916F002B7F20936F0067
:1007500002C024E026BB00918C0110918D012091F4
:100760008E0130918F01060F171F281F391F00932C
:100770008C0110938D0120938E0130938F0181E0C5
:100780008093860180916F00846080936F001F9139
:100790000F91089561E070E080E090E00C949D037B
:1007A0006FEF7FEFCB010C949D031F920F920FB65A
:1007B0000F9211248F939F93EF93FF93E8E8F0E05B
:1007C00080819181985B9183808381E0809368012F
:1007D000FF91EF919F918F910F900FBE0F901F90FF
:1007E00018958091710181110EC081E08093710193
:1007F0008FE087BD85E088BD84B5836284BD85B503
:10080000896085BD559A089506C0109268012091AF
:1008100068012223E1F30197C0F70895CF93DF9396
:10082000CDB7DEB7CC55D1090FB6F894DEBF0FBEF9
:10083000CDBF8CE5ECE0F1E0EE24E394F12CEC0E7E
:10084000FD1ED70101900D928A95E1F780E8809313
:100850006100109261000E94F10300910201109169
:10086000030120910401309105014091060150914E
:100870000701609108017091090180910A0190912E
:100880000B010E94740280910001909101019093EC
:100890007D0180938B0188EC90E00E940404DE2CA3
:1008A000CF2C7E018DE5E80EF11C69817A818B8168
:1008B0009C810E944D0260E876E988E990E00E9400
:1008C00013038CE291E00E9404040D2D1C2D0CC03A
:1008D000F80161917191819191918F010E944D0276
:1008E0008CE291E00E9404040E151F0589F784EF45
:1008F00091E00E9404040E9455030E94EE0260E011
:100900007DE780E090E00E944D0260E070E0CB0166
:100910000E9413030E94EE0288EE93E00E940404FA
:10092000C4CFA1E21A2EAA1BBB1BFD010DC0AA1F3A
:10093000BB1FEE1FFF1FA217B307E407F50720F048
:10094000A21BB30BE40BF50B661F771F881F991FC3
:100950001A9469F760957095809590959B01AC010C
:10096000BD01CF010895052E97FB16F4009407D022
:1009700057FD0DD00E94910407FC09D07EF490959C
:100980008095709561957F4F8F4F9F4F089550953B
:100990004095309521953F4F4F4F5F4F0895F89404
:0209A000FFCF87
:1009A2000A033200007D0000800C000010270000C6
:1009B200D92B00003831000024340000873A0000AF
:1009C200B1410000BD490000204E0000204E000051
:1009D200BD490000B1410000873A00002434000004
:1009E20038310000D92B000010270000204E0000F3
:1009F2001027000088130000102700003831000083
:080A0200873A0000204E0000BD
:00000001FF
